:10000000DD29A501A400B3172730A3001030142068
:100010000330A300E8301420A30164301420A301AE
:100020000A30142024081F28A2002508A100240853
:10003000A0009B212008031DB313B31B0800303E12
:1000400022280408A2008316051183120930A30098
:1000500003103520A20CA30B2928031435200330EC
:10006000A100E83059210314D82903183A280000C8
:1000700005113C2805153C280030A10062305929A3
:10008000A501A400B3172730A3001030532003307C
:10009000A300E8305320A30164305320A3010A30A9
:1000A000532024085E28A2002508A1002408A000EF
:1000B0009B212008031DB313B31B0800303EA6008C
:1000C000360884000930A70003106B20A60CA70B8C
:1000D000652803146B288413B31D7A2800083404A0
:1000E000331D34068000841700083404031C3406D2
:1000F0008000852800083404031C340633193406B4
:100100008000841734098005852800308A00330D6B
:100110000639A0009220A10000308A00200A922017
:1001200000005929963E03188A0A82000134893456
:1001300003342934003450340C34ED342C08A0003E
:100140002D08A1000130A200A3016400CE20031CF1
:10015000B928A20BA528FF30A3070318A528A007DC
:10016000031CA107031C08006430A2000030A30098
:10017000A528E920A801A2010930A300EA20CE2089
:100180000318A80AAB1EA801A20CA30BBE28AB1A29
:10019000A213A20DEA2003142208080036088400E6
:1001A000340884178004841300052B1B3406FF3E9B
:1001B0000800A400290803140319D829D321031C1B
:1001C0000800A0002408840020088000A40AA903D5
:1001D000DA2833172B081F39003EA1002A08043EF5
:1001E0000318A10A331F59293313A0000310A10CCF
:1001F000A00C0310A10C200C5929B31329080319D2
:10020000B3171030A8000301A40DA50D0318013089
:1002100020212808031D03290800B3132908031906
:10022000B3170430A800250E1A2125081A21240E20
:100230001A2124080F39F63E0318073E0A3E2029EA
:10024000A000A8030319B313290803192A292802B7
:10025000031808002008031DB313B31B0800303E29
:10026000D3298001840AFF3E031D3129D829831632
:100270001C141A0883169B0AD829030183169A00B6
:100280001C1555309D00AA309D009C149C184629D1
:100290001C119B0AD829A301A200FF30A207031C4E
:1002A000A307031CD8290330A100E33059214D29AD
:1002B000A101F43EA000A109FE30031C6229A007A1
:1002C00003185F29A0076400A10F5F290000201810
:1002D000692920186B290800A000A11BCD21200846
:1002E000D829A20002307D29A20003307D29A20076
:1002F00006307D29A20004307D29A80023082102B0
:10030000031D842922082002043003180130031938
:1003100002302805031DFF30D829A2002008A600BE
:100320002408A0002608A4002108A6002508A10092
:100330002608A5009D29A501A4011030A600210DC5
:10034000A40DA50D2208A4022308031C230FA50257
:100350000318B1292208A40723080318230FA507AF
:100360000310A00DA10DA60B9F292008D82910303D
:10037000A800A101A001A70CA60C031CC5292208F6
:10038000A00723080318230FA107A10CA00CA50C9C
:10039000A40CA80BBB292408D829A009A109A00AEC
:1003A0000319A10A0800840031088A00300882007D
:1003B0008313031383126400080088308B008316B4
:1003C00075308F0083120730990083161230850034
:1003D00052309F00831285309F00203084006030AF
:1003E0003121A0308400203031216E30E4006400DF
:1003F0008330640203180C2A640883169B0083125E
:100400003721E8000530B6002030B4000630B300D4
:1004100068085F20E40FF7298316FF309B008312E2
:100420003721E5008316FD309B0083123721E00061
:10043000E1016400E51C382A0730A300D0304C21CC
:10044000E4016400263064020318302A640883162D
:100450009B0083123721E80068082220E40F212A3C
:100460000730A300D0304C21FE3022200130222062
:100470000530B6001030B4005430AA002030AB0074
:10048000FA30AC00AD019E20031C142F873C031DE5
:10049000432A0B30A9009E30B000B1013830D9207A
:1004A000031C142F8730E300E40164000A30640267
:1004B0000318632A6408383E84000008DA005A08EA
:1004C000E307E40F552AE309E30A7F30E3056400FC
:1004D00042086302031D382A0530B6001030B4000C
:1004E0005430AA002030AB00FA30AC00AD019E20A1
:1004F000031C142FAA3C031D772A0B30A9009E3041
:10050000B000B1014330D920031C142FAA30E300FE
:10051000E40164000A3064020318972A6408433E29
:1005200084000008DA005A08E307E40F892AE30987
:10053000E30A7F30E30564004D086302031D6C2A63
:100540003908A600A7010230A200A301B721E900E3
:1005500007303A05E4006408A600A7018030A20035
:10056000A301B721DA002508DB003B085A07D800B1
:100570005B080318013ED9003C08A600A7018030A3
:10058000A200A301B721DA002508DB003D08DA0745
:100590000318DB0A00305A02CE000830031C013E6B
:1005A0005B02CF006400CF1FD82A2D30E200DA2A88
:1005B0002B30E2004F08A1004E086C21CE0021082C
:1005C000CF004E08A6004F08A700C430A200093093
:1005D000A300B721CE002508CF000230A3000030D1
:1005E0008D21CE002108CF004E08A0004F08A100A9
:1005F0006430A200A3019B212408DA002508DB0057
:100600005A08A0005B08A1000A30A200A3019B21A8
:10061000E4004E08A0004F08A1006430A200A3012E
:100620009B21CE002108CF004E08A6004F08A7004E
:100630006430A200A301B721DA002508DB005A08C4
:10064000A0005B08A1000E30A200A3019B21D600F0
:100650002108D700640062082B3C031D482B560874
:10066000D00757080318013ED1075008A0005108D1
:10067000A100A30164307A21031D482BE00A03196D
:10068000E10A6430D0020030031C013ED102352B58
:10069000640062082D3C031D752B5608D2075708CD
:1006A0000318013ED3075208A0005308A100A3017C
:1006B00064307A21031D752B0130E0020030031CE9
:1006C000013EE1026008A0006108A100A301013021
:1006D0007421031D6E2B0130E000E1016430D20271
:1006E0000030031C013ED302532B6008A0006108B8
:1006F000A1002730A3000F307721031D832B0F307B
:10070000E0002730E1006008A0006108A10064302B
:10071000A200A3019B21D4002108D5006008A000FD
:100720006108A1006430A200A3019B212408DA0023
:100730002508DB005A08A0005B08A1000A30A200CF
:10074000A3019B21D6002108D700640020303F027E
:100750000318B42B3F08203CDC000030031CFF3E94
:10076000DD002D30E600BD2BE0303F07DC00FF3020
:100770000318013EDD002B30E6006400203040020B
:100780000318CC2B4008203CDE000030031CFF3E49
:10079000DF002D30E700D52BE0304007DE00FF30D2
:1007A0000318013EDF002B30E700640065185E2C63
:1007B000640066082D3C031DFE2B5C08A6005D0846
:1007C000A7001230A200A301B721DA002508DB0040
:1007D0005A08A0005B08A1000A30A200A3019B21D7
:1007E000DA002108DB005A08203CDC005B08031C0F
:1007F000013E003CDD002B30E6001B2C5C08A6000F
:100800005D08A7001230A200A301B721DA00250875
:10081000DB005A08A0005B08A1000A30A200A30177
:100820009B21DA002108DB0020305A07DC005B083E
:100830000318013EDD00640067082D3C031D412CB8
:100840005E08A6005F08A7001230A200A301B7212E
:10085000DA002508DB005A08A0005B08A1000A3076
:10086000A200A3019B21DA002108DB005A08203CEA
:10087000DE005B08031C013E003CDF002B30E7007C
:100880005E2C5E08A6005F08A7001230A200A3013C
:10089000B721DA002508DB005A08A0005B08A10098
:1008A0000A30A200A3019B21DA002108DB002030DE
:1008B0005A07DE005B080318013EDF00FE302220ED
:1008C0008030222069080120203022206400651F2A
:1008D0008B2C5808A0005908A1000A30A200A301DF
:1008E0009B21DA002108DB005B08A5005A080220E2
:1008F0002E3022205808A0005908A1000A30A2007A
:10090000A3019B212408DA002508DB005B08A50071
:100910005A080220952C5508A500540802202E30B4
:1009200022205708A500560802202530222020301A
:100930002220620822204F08A5004E0802202E30F7
:100940002220640801202030222020302220FE3086
:100950002220C0302220660822205D08A5005C0805
:1009600002204830222020302220670822205F0801
:10097000A5005E0802204C30222020302220533077
:1009800022200230A9004808A400A5012130B000AF
:10099000B1010D2120302220203022206400651971
:1009A000172D0530A300DC304C21FE302220013011
:1009B0002220FE302220803022200130E40064001A
:1009C000093064020318F42C0230A9006408383E90
:1009D00084000008DA005A08A400A5012130B00004
:1009E000B1010D21E40FDF2CFE302220C030222087
:1009F0000130E40064000930640203180F2D023056
:100A0000A9006408433E84000008DA005A08A400E4
:100A1000A5012130B000B1010D21E40FFA2C053001
:100A2000A300DC304C21FE30222001302220640063
:100A3000E51A5C2D0530B6002030B4000630B30056
:100A400044305F2041305F2054305F2041305F20D0
:100A50002C305F2054305F2049305F204D305F20C4
:100A600045305F202C305F20690840202C305F200B
:100A700062085F202C305F204F08A5004E084120FF
:100A80002C305F205908A500580841202C305F20E9
:100A900066085F202C305F205D08A5005C084120BF
:100AA0002C305F2067085F202C305F205F08A50096
:100AB0005E0841200D305F206400E519D32D05301C
:100AC000B6002030B4000630B30044305F2041301F
:100AD0005F2054305F2041305F202C305F20543045
:100AE0005F2049305F204D305F2045305F202C3043
:100AF0005F20873040202C305F20E40164000B3001
:100B000064020318942D0530B6002030B40006307E
:100B1000B3006408383E84000008DA005A08402018
:100B20002C305F20E40F7E2D0530B6002030B4005D
:100B30000630B3000D305F2044305F2041305F202D
:100B400054305F2041305F202C305F2054305F20D4
:100B500049305F204D305F2045305F202C305F20D2
:100B6000AA3040202C305F20E40164000B30640286
:100B70000318CB2D0530B6002030B4000630B3008A
:100B80006408433E84000008DA005A0840202C30F4
:100B90005F20E40FB52D0530B6002030B4000630DC
:100BA000B3000D305F20DE255408A0005508A100D9
:100BB000A30100307121031D102E382A9F146400F8
:100BC0009F1CE32DDF2D1E08D50083161E088312FF
:100BD000D40006305407DA0055080318013EDB0044
:100BE0005A08A0005B08A100AA30A200A3019B2123
:100BF000DA002108DB0001305A02D4000030031C67
:100C0000013E5B02D5005408A0005508A100A301D5
:100C100005307721031D0F2E0530D400D5010800C3
:100C20002630E40064004A3064020318212E640870
:100C300083169B0083123721E80068082220E40F06
:100C4000122E0330A300E8304C21DE255408A10009
:100C5000043C031C472E5508031D472EA10D3626C4
:100C6000A000211036268A002008820006308A0063
:100C700021083D3E03188A0A820006347034063487
:100C8000483406344F340634563406346134212E49
:100C90006400651C4D2E65104E2E6514C22E640036
:100CA000651D542E6511552E6515C22E6400E51C78
:100CB0005B2EE5105C2EE5147C30222009302220CA
:100CC000C22E6400651E6A2E65127C3022208C3094
:100CD00022206F2E65167C3022209D302220C22ECD
:100CE0004A30E40064006E3064020318812E640808
:100CF00083169B0083123721E80068082220E40F46
:100D0000722E0330A300E8304C21DE255408A100E8
:100D1000043C031CA72E5508031DA72EA10D9626E3
:100D2000A000211096268A002008820006308A0042
:100D300021089D3E03188A0A82000634C234063414
:100D4000A8340634AF340634B4340634BB34812EB0
:100D50006400E51DAD2EE511AE2EE515C22E0F3057
:100D6000E0002730E100C22E6400E51EB92EE51236
:100D7000BA2EE516C22E6400651FC02E6513C12E63
:100D80006517C22EFE30222001302220FE302220A4
:100D9000803022204F3022207030222074302220D8
:100DA000693022206F3022206E3022202030222015
:100DB0005508A50054080220203022204F30222060
:100DC0006B302220FE302220C030222043302220EF
:100DD0006F3022206E30222066302220693022209F
:100DE00067302220203022203D3022200830A90008
:100DF0006508A400A5012130B000B101FD208316D3
:100E0000FF309B00831265083E218316FD309B0056
:100E1000831260083E210B30A300B8304C21FE3015
:100E2000222001302220382AFE30222001302220C8
:100E3000FE302220803022204E3022206F302220AF
:100E40002030222042302220433022204D302220E8
:100E50002030222044302220613022207430222091
:100E600061302220213022200330A300E8304C21C1
:020E7000382A1E
:02400E009C3CD8
:104200007C009D00FE008000420043004D00200025
:10421000470061007500670065002000200056001F
:1042200033002E0030003000FE00C0007700770021
:1042300077002E003100350030006D0070006700FF
:104240002E0063006F002E0075006B00FE008000E2
:10425000540065006D0070003D00550020002000F6
:10426000530070006C006100730068003D00440062
:10427000FE00C0004800650078004400690073003B
:104280003D00520020004C00690067006800740087
:104290003D004C00FE00800048006500780054009E
:1042A00078003D005500200020004E006F00720095
:1042B000540078003D004400FE00C000520073002E
:1042C000740053006F0063003D005200200058004E
:1042D000740053006F0063003D004C000D004D0062
:1042E000530047002C00420043004D0020004700CF
:1042F00061007500670065002000440061007400E3
:0443000061000D004B
:00000001FF
